:020000040800F2
:10000000C01B0020A9010008E1100008C108000879
:1000100000000000000000000000000000000000E0
:10002000000000000000000000000000291400088B
:100030000000000000000000E3100008291500087F
:10004000BB010008BB010008BB010008BB010008A0
:10005000BB010008BB010008BB010008BB01000890
:1000600000000000BB010008BB010008BB01000844
:10007000BB010008BB010008BB0100080000000034
:10008000BB010008BB010008000000002D1600089D
:1000900061160008C9160008ED160008BB0100082B
:1000A000BB010008BB010008BB0100084D17000898
:1000B000DD17000800000000000000000000000044
:1000C000BB01000800000000BB01000800F002F8BE
:1000D00000F03EF80CA030C8083824182D18671E10
:1000E000A246AB4654465D46AC4201D100F030F822
:1000F0007E460F3EB6460FCC0126334200D0FB1A97
:100100003343A246AB461847543D0000743D0000FF
:10011000103A02D378C878C1FAD8520701D330C850
:1001200030C101D504680C60704700000023002432
:1001300000250026103A01D378C1FBD8520700D31E
:1001400030C100D50B6070471FB51FBD10B510BD85
:1001500000F0A1F91146FFF7F7FF02F0A1FA00F055
:10016000B9F903B4FFF7F2FF03BC00F0BFF90000D8
:1001700070B505460C46164602E00FCC0FC5103E82
:10018000102EFAD2082E02D303CC03C5083E042E4B
:1001900007D301CC01C5361F03E021782970641C08
:1001A0006D1C761EF9D270BD07488047074800478E
:1001B000FEE7FEE7FEE7FEE7FEE7FEE70448054947
:1001C000054A064B704700003D150008CD000008A9
:1001D000C0130020C01B0020C0170020C017002043
:1001E000F8B5042A2CD3830712D00B78491C03706E
:1001F000401C521E83070BD00B78491C0370401C17
:10020000521E830704D00B78491C0370401C521EF9
:100210008B079B0F05D0C91ADF002023DE1B08C9FE
:100220000AE0FFF7A5FFF8BD1D4608C9FD401C46C2
:10023000B4402C4310C0121F042AF5D2F308C91A87
:10024000521EF0D40B78491C0370401C521EEAD495
:100250000B78491C0370401C012AE4D40978017012
:10026000F8BD01E004C0091F0429FBD28B0701D5AA
:100270000280801CC90700D00270704700290BD093
:10028000C30702D00270401C491E022904D3830711
:1002900002D50280801C891EE3E70022EEE70022DF
:1002A000DFE7704770477047F0B5FF252D04C6099A
:1002B000C209FF2704462E400137CB093E43484080
:1002C0002A402B400746002A6BD0002B69D0AA4257
:1002D00067D0AB4265D0002800DA32460125ED0533
:1002E00029432C4309022002090AD21A4B0C7F240D
:1002F000E31A434C000A7C44E35C7D242404121975
:1003000014145B00A218884201D3521C00E0400084
:1003100049420C465C4324115C43DB016415E3183D
:10032000040A5C43C502200D0C4644436419250AA7
:100330005D432303EC0C0D46654300030019EB18E5
:100340004C42A34201D35B18401CD4052018002B5B
:1003500007D05B00C91804D3401C002901D1400814
:1003600040003F2189048A4209D3002A08DC110693
:10037000090F04D0032149074018C00FC007F0BD82
:1003800001224100120689187F2252069142F6D2BC
:1003900005214907C84201D59010F0BDFF20C005D6
:1003A000F0BD002F00DA32461648AA4207D2AB420F
:1003B00005D21902090E17D0F80FC007F0BDFF25AE
:1003C00063002D06AB42F9D84900A942F6D8AB42EA
:1003D00001D1A942F2D0A94201D1002101E061007E
:1003E0004908D0050843F0BD1102090EFBD0FF20DB
:1003F0000243D005F0BD0A460146104654E700000E
:100400003A3800000000C07F0102C21504D0012369
:10041000DB071943002A0ADB9E239A1A02D40846F6
:10042000D0407047FF2241001206914201D90020BE
:100430007047C017C04370471F22030C02D10F2220
:1004400000041CD0030E01D10002083A030F01D1B1
:100450000001121F830F01D18000921E002801DBD2
:100460004000521ED2055118021251181922904014
:1004700004D3491C002801D14908490008467047A7
:10048000C10FC90700D04042012292071143D3E7B0
:1004900001218907D0E7754600F024F8AE46050033
:1004A00069465346C008C000854618B020B5FFF71E
:1004B00085FE60BCB64600260027C0C5C0C5C0C5C5
:1004C000C0C5C0C5C0C5C0C5C0C5403D490849007C
:1004D0008D46704710B50446C046C0462046FFF71B
:1004E00040FE10BD004870479000002001491820D0
:1004F000ABBEFEE72600020070470000B0B588B032
:10050000974802F091FD40F2005002F08DFD00246A
:10051000204601F0C1FA01AD40F200102883AC760C
:100520000E4901910E49891C039140F2004104914A
:10053000029042F20000069008200590204601F04B
:10054000A3FA2046294601F0D1FA204601F006FB25
:10055000204601F091FA08B0B0BDC0464C240140DD
:100560003C01002070B514460D460646200407D015
:10057000B0B200F007F82870641E6D1C761CF5E719
:1005800070BD000070B5044600F054F9A020214D64
:10059000A847214EB047200AA847B047E0B2A84775
:1005A000B04700F047F9A120A847B047002000F06D
:1005B00089F9044600F05EF9204670BD70B5144616
:1005C0000D460646200407D02978B0B200F006F8A0
:1005D000641E6D1C761CF5E770BD0000F8B50C4676
:1005E000054600F027F9A0200A4EB0470A4FB84749
:1005F000280AB047B847E8B2B047B8472046B047E6
:10060000B84700F037F90A20F8BC02BC8E4600F06B
:10061000B9B8C046290900088D090008F0B50B4D8E
:1006200000210B4A0B4B0C4684420DD0165D7540E1
:100630000E46072E06D86F08ED0700D05F403D46F6
:10064000761CF6E7641CEFE7A8B2F0BDFFFF0000E0
:10065000A10A002001A00000984800218170704785
:10066000F0B587B040F2005011303C4CA04740F24A
:1006700000501230A0473A48A04740F20050A0472F
:100680000620059002F0DAFB09200690C00603243C
:1006900004940025F32321462A4601F0C1FF314886
:1006A00021462A46234601F0BBFF01F01FF9FFF760
:1006B00025FF012640F20010314601F0ADF902207D
:1006C0000190314601F0A8F907200390410430461B
:1006D00001F02CF9284601F0FDF8284601F080F9D8
:1006E00008210291304601F0D5F805241E4F284616
:1006F00029462246B847304631462246B8470425A7
:10070000019829462246B847049821462246B84710
:100710002846059D29462246B8472046039F39466C
:100720002246114B98472846029922460E4DA8476B
:10073000384606992246A84701F0EEF801F0ECF899
:1007400001F098F801F0E0F8304601F053F9304636
:1007500007B0F0BC02BC8E4601F04CB9293000084D
:1007600009060000000400485519000838B1044982
:1007700041430F204003B1FBF0F10A20484370478A
:10078000E880000081B00090034800990160016892
:100790000029FCD101B07047E40A002081B000902C
:1007A000009801B07047F8B505460920C4062046F8
:1007B00040F6000101F029FF204641F2000101F05E
:1007C00024FF00270126082F20D02846F840C00724
:1007D00005D0204648F2000101F019FF04E0204650
:1007E00048F2000101F011FF3046FFF7D7FF204625
:1007F00040F6000101F00BFF3046FFF7CFFF204627
:1008000040F6000101F001FF7F1CDCE701252846CE
:10081000FFF7C4FF204641F2000101F0F8FE284630
:10082000FFF7BCFF204641F20001F8BC04BC96462D
:1008300001F0EBBEF8B500F043FE814C01262046E6
:10084000314601F0E4FE02252046294601F0DFFE94
:1008500004273846FFF7A2FF2046314601F0D5FEB7
:100860003846FFF79BFF20462946F8BC04BC964655
:1008700001F0CBBEF8B500F023FE714C02252046F6
:10088000294601F0C2FE01262046314601F0BDFE98
:1008900004273846FFF782FF2046294601F0B7FEBD
:1008A0002046314601F0B3FE3846F8BC02BC8E4605
:1008B000FFF774BF014880787047C046F000002001
:1008C000FEE70000FEB5009000F0F4FD00210226D6
:1008D000012001900C46019D07291CD8584F38462D
:1008E0000291314601F091FE3046FFF757FF38463E
:1008F000314601F08CFE3846294601F08CFE274631
:1009000004462846FFF74AFF0299601E844178009A
:100910000419491CE0E7009810B100F08DFD01E0DA
:1009200000F0AAFDE0B2FEBDFEB5044600F0C8FD31
:1009300043480226314601F068FE0027012001905D
:10094000072F1FD860B2002802943D4D284603D4DB
:10095000019901F05AFE02E0019901F058FE30467B
:10096000094CA0472846314601F051FE3046A047C9
:100970002846314601F049FE3046A0477F1C029CC4
:100980006400DDE7FEBDC0469D07000870B500F0BD
:1009900091FD2B4C0221204601F039FE012528460D
:1009A000FFF7FCFE00262046294601F034FE30B158
:1009B000701CFA2E0646F6D3FFF75CFF04E0022116
:1009C000204601F022FE0025284670BDC046C046E4
:1009D000F8B5394802F028FB384801250024934E29
:1009E0002946224648F20003B0470326904F334879
:1009F0002146324648F20003B847304848F2000129
:100A000001F003FE2C48C01C02F00EFB0C482946E6
:100A100022462B46854FB8470948214632462B4689
:100A2000834FB84702270648294622463B467F4D5A
:100A3000A8470348214632463B467D4CA047F8BDB7
:100A400000140048F8B5774802F0EEFA764C00251D
:100A500001261023754F204629463246B8472023E9
:100A6000204629463246B84740232046294632468A
:100A7000B8478023204629463246B847F8BDC046CD
:100A8000B0B50D4802F0D0FA0C4C012100252046EB
:100A90002A4642F2000301F0C3FD03222046294604
:100AA00042F2000301F0DBFD204642F20001B0BC3F
:100AB00004BC964601F0A9BD1305000000080048DB
:100AC00070470000F0B585B0564802F0ADFA564CBC
:100AD000012103910227554D20463A46049740F2E2
:100AE0000013A84700210291032520462A460195BC
:100AF00040F200134E4EB047204640F200114D4ADE
:100B000090472046039E31463A4640F20023F14F7B
:100B1000B8472046029F39462A4640F20023444DFA
:100B2000A847204640F20021424A904720463146DD
:100B3000049E324640F20043E64DA847204639461F
:100B4000019A40F200433A4DA847204640F2004146
:100B5000384A904720460399324640F60003DD4D5F
:100B6000A84720463946019D2A4640F60003304EEC
:100B7000B047204640F600012E4A90472046039E8B
:100B80003146049A41F20003D24FB84720460299F9
:100B90002A4641F20003FB4FB847204641F20001CC
:100BA000F94A904720463146049E324642F20003FD
:100BB000F34FB847204602992A4642F20003F14F0C
:100BC000B847204642F20001EF4A90472046039F73
:100BD0003946324644F20003E94EB0472046029EB1
:100BE00031462A4644F20003E64DA847204644F227
:100BF0000001E54A904720463946049A48F200032E
:100C0000DF4DA84720463146019A48F20003DD4DEA
:100C1000A847204648F20001DB4A05B0F0BC08BCFA
:100C20009E461047120500000004004821260008D7
:100C30005F2600080B2600080C48006840F2E831E7
:100C4000B0FBF1F0401E010E00D0FEE70849094A52
:100C50005060094803680B40032189075918016057
:100C600000209060072010607047C04604000020FC
:100C7000FFFFFF0010E000E020ED00E0F0B587B0DE
:100C800037480021017041600E460191354940F21C
:100C900010608847344D35492846884703AC3449AD
:100CA00020468847472002902080324805900496CD
:100CB000314A2846214690470127304A284639467E
:100CC00000979047142002212D4A90472D4928462D
:100CD000884740F21060401C224988472A4E30461F
:100CE0002249884703AD2846214988470298288031
:100CF00020480590019C0494304629461E4A90479E
:100D0000304639461D4A90471520032529461C4A7E
:100D1000904730461B49884740F21060801C1149BB
:100D200088471A4E30461149884703AF3846104964
:100D3000884717483880174805900494304639464C
:100D40000D4A9047304600990C4A90471620294694
:100D50000B4A904730460B49884707B0F0BDC04664
:100D6000F00000202930000800400140C530000894
:100D700011320008E703000039310008ED310008A6
:100D8000692D00082F31000800440140004801404F
:100D90001F1C00000F270000FEB502901C20022738
:100DA0003946009701F0E0FF744802F03DF9092050
:100DB000C50601240426019628462146324601F044
:100DC000F9FB284639462246334601F029FC002724
:100DD000284639462246334601F041FC082628467B
:100DE0002146324601F0E6FB28460099224633466A
:100DF00001F016FC284639462246334601F02FFC06
:100E0000144802F011F9144C204602F057FA20461B
:100E1000029902F021FA2046394602F0C9FA20462A
:100E2000394602F0DAFA2046394602F0ACFA20469A
:100E3000019902F0B5FA2046314602F0C6FA204682
:100E400002F056FA0521204603B0F0BC04BC9646D9
:100E500002F06CBA1107000000440040F8B51B4CCA
:100E6000204602F0E1F8204602F0DEF8184F012497
:100E70004025434E3846214622462B46B0470026A1
:100E800003220092384631462B4601F0E8FB3846F3
:100E9000294601F0BAFB02228025384621462B461E
:100EA000374FB8470A4F38463146009A2B4601F073
:100EB000D6FB3846294601F0AAFB8848314622462F
:100EC00044F200032E4CA047F8BDC04616050000B2
:100ED0000014004821260008FEB5284802F0A4F8B6
:100EE0000920C40601260025254F204631460296DA
:100EF0002A4640F60003B8470322019220462946BD
:100F000040F600031F4FB847204640F600011E4A36
:100F10009047204631462A4641F20003184EB0471A
:100F200020462946019F3A4641F20003154EB0473C
:100F3000204641F20001144A9047204602992A4671
:100F400048F200030E4EB047204629463A4648F282
:100F500000030C4DA847204648F200010A4A90477A
:100F6000204640F60001084A9047204641F2000121
:100F7000054A03B0F0BC08BC9E46104711050000AE
:100F8000212600085F2600080B26000802480021E1
:100F90004170FFF765BBC0463C010020F0B58FB043
:100FA00007A82021FFF77BF90024022520462946C7
:100FB00000F092FD0028F9D000200221059000F0F9
:100FC00081FD4A203E493F4B5A2805D00A184A3A2B
:100FD00012881A52801CF7E701223A494A70C54B21
:100FE0003948C01C04900A2003909A480446C8342B
:100FF0000294283001900692104600285DD088792E
:1010000040B10020887101204821082200F050F9E9
:10101000B84B2C49187800284DD0059919700498C0
:10102000082914D08B0007AC0022E250E3181825E1
:101030001446042A07D0F8272F40865CBE40341996
:10104000F835521CF5E71C60001D491CE8E70898BC
:10105000039BB0FBF3F00999B1FBF3F1194AD0619E
:1010600011620798B0FBF3F07A4988600199029AFF
:10107000059B062B18D00860069C9C401568A8426A
:1010800002D8156CA84208D2104EB57825433446D4
:10109000A5701031121D5B1CEBE70C4DAD782C4296
:1010A000F7D0A543094CF3E706490698087205985E
:1010B0004870904BA1E748789FE70FB0F0BDC0465D
:1010C0003E010020240200207301002000000020C7
:1010D000024842F2000101F09CBAC04600080048F4
:1010E00070477047F0B587B00024594D2046294617
:1010F00040F20012FFF736FA287808B1072802D329
:10110000534906200870697840F2C812514B995033
:10111000E97840F2D01299504F4908700695062C94
:1011200000D187E0611D685C08B1642801D300200C
:10113000685422461532A95C09B1642901D3002103
:10114000A9540194A200434BD31840F2182299509D
:1011500040F2D8115850C82000261E5040F2081006
:101160001E5040F248115E5040F288129E509A186C
:1011700004925918059118180290C833039303205C
:10118000C4431822304631463346A4B1069D2F1978
:10119000BD257D5D9540AE198D257D5D9540281856
:1011A0005D257D5D954069182D257D5D9540EB1889
:1011B000083A641CE9E7029A1160039A1360059AE1
:1011C0001060049A1660254A934202D3254CA3422C
:1011D00002D9244B039C23609142019C1C4D02D3F5
:1011E000204FB94202D902990A6011468B4203D2BC
:1011F000029A1360039A116040F2F411884202D3FC
:10120000174A904202D91648059A10608E4202D3BE
:10121000134A964203D9049A116040F2F416B04280
:1012200003D204990860059806600698001D069090
:10123000641C74E725200649085C40F25822054BDF
:1012400098502720085C40F25C21585007B0F0BD50
:10125000A00500208002002001000020E02E0000F8
:10126000905F0100D0DD060070B56E4C10210E4E6F
:101270002046B0470D4D287020212046B0476870A9
:1012800040212046B047A87080212046B047C000CA
:10129000A978890001436878400008432978014310
:1012A0000F20884370BDC0462B1400083801002071
:1012B000B0B5104B00251D700F4B1D700F4C6271A7
:1012C0002571E17003236370207090000C4A107048
:1012D000090AA170401D0B4908700620FFF79EF90E
:1012E000A071000AE07108212046B0BC04BC9646FB
:1012F00000F002B97201002070010020A10A002054
:10130000A00A002071010020B0B5464C07283DD846
:10131000820001A39A18974600F00EB800F012B8A8
:1013200000F016B800F01AB800F01EB800F022B8AD
:1013300000F051B800F024B82046012955D140F200
:1013400000114DE02046012952D140F2002147E032
:10135000204601294FD140F2004141E020460129B9
:101360004CD140F600013BE02046012949D141F231
:10137000000135E02046012946D142F200012FE06C
:101380002046012943D148F2000129E0394D204689
:1013900040F20011A847204640F20021A84720460D
:1013A00040F20041A847204640F60001A8472046E9
:1013B00041F20001A847204642F20001A84720461A
:1013C00044F20001A847204648F200012A46B0BC7A
:1013D00008BC9E461047204601291BD144F200015B
:1013E000B0BC04BC964601F012B940F2001113E003
:1013F00040F2002110E040F200410DE040F6000113
:101400000AE041F2000107E042F2000104E048F284
:10141000000101E044F20001B0BC04BC964601F0BA
:10142000F4B8C04600040048704780B501F0F3F8F6
:10143000411E884180BD000070B52D4C02250D4E27
:1014400020462946B04700F03BF801212046B0472E
:101450002846FFF7A3F92046294601F0D8F8284688
:10146000FFF79CF920462946324670BC08BC9E46D0
:101470001047C0460B260008B0B51D4C022520467B
:10148000294601F0C2F800F01BF80121204601F0C6
:10149000BEF82846FFF782F92046294601F0B7F842
:1014A0002846FFF77BF920462946B0BC04BC964687
:1014B00001F0ABB8EE48002101230A4601F0B0B8B4
:1014C00070B5EB4C00250126204631462A463346AE
:1014D00001F0A6F8032220462946334601F0BFF862
:1014E000044848F2000170BC04BC964601F08DB877
:1014F0000014004800080048F8B50C46009000258C
:10150000C54E084FA5420CD00098415D304601F011
:10151000CFFE3046394601F0F8FE0028F9D06D1CA8
:10152000F0E7F8BD060700000348016811B1016843
:10153000491E01607047C046E40A002030B43348B9
:10154000026801210A43026002689207FCD54268E2
:101550002F4B1340436042682E4B13404360026898
:101560002D4B13400360C26A0F239A43C262026B81
:1015700040F203139A4302630A04036B9343036329
:10158000CA07036B93430363426B8A43426300229F
:10159000826002680A430260204B022204685D1EDA
:1015A0009D4202D214402B46F8D003689B0700D41A
:1015B000FEE71B4B1C680725AC431C601C681443EA
:1015C0001C6043684360436843604368436043680A
:1015D000144C1C4044604368134C1C4344600B068D
:1015E00004681C43046003689B01FCD54368032422
:1015F000A343436043681343436042681207FCD52A
:10160000C806002130BC01F0E3BBC0460010024018
:101610000C00FF08FFFFC277FFFFF2FEFF0400008F
:1016200000200240FFFFC2F70000040810B50A4C7A
:101630000121204601F0E2FD68B10121204601F0C0
:10164000D9FD0021204601F03BFD0448006810BC94
:1016500002BC8E46004710BD00200040140200204E
:10166000F8B5164D01242846214601F0C7FD012892
:1016700003D10121284601F0BDFD3149203100226E
:101680000F4B1646062E13D0985D0F46183F28B113
:1016900038680D68A84203D2401C05E03A6004E0B7
:1016A00008488455002098553860091D761CE9E7E4
:1016B0002349486808B1401E4860F8BD0040014019
:1016C000480200205A02002010B5074C0121204694
:1016D00001F094FD012806D10121204610BC04BC74
:1016E000964601F087BD10BD00440140B0B5134DD2
:1016F00001242846214601F081FD012803D1012162
:10170000284601F077FD0E4884700178042901D83D
:10171000491C02E00B490C70002101700A490A784B
:1017200022B14278092A04D8511C00E000214170FE
:10173000B0BD00220A704270B0BDC04600480140F2
:10174000F00000202A02002025020020B0B51D4C28
:10175000324D2046294601F007FE30B11A48006894
:1017600080472046294601F0EBFD184D20462946CA
:1017700001F0CBFD012806D12046294601F0BDFD30
:10178000114800688047124D2046294601F0ECFDC3
:1017900030B11048006880472046294601F0D0FD4E
:1017A0000D4D2046294601F0DFFD48B1094800688B
:1017B000804720462946B0BC04BC964601F0C0BD17
:1017C000B0BDC046003801400C02002003070000F5
:1017D000070007071002002006000607B0B50E4CF0
:1017E0000E4D2046294601F0BFFDA0B120462946F6
:1017F00001F0A6FD204601F057FD09490A78531C67
:101800000B708A18D0704878DAB2824203D3012074
:10181000887000200870B0BD004400400500050736
:1018200070010020B0B50020064CA047064D28608E
:101830000120A04768600220A047A8600320A047BD
:10184000E860B0BD012F000828010020B0B5084CA9
:1018500080252046294600F0DAFE2046294600F081
:10186000D4FE20462946B0BC04BC964600F0CFBE4C
:10187000001400486748016808220A4302600168B2
:101880000907FCD4016804220A4302600168490781
:10189000FCD4704702280ED0012818D10F20000573
:1018A0000B4A136883431360090509180140106847
:1018B00008431060704703200005054AD36883433E
:1018C000D360090509180140D0680843D06070470B
:1018D0002C240140411E8841C0024E490A6840F64E
:1018E00000039A43101808607047C04610B5054CB5
:1018F000204601F0ADFB204610BC02BC8E4601F034
:101900009DBBC046090300004248016840F2001236
:101910000A4302607047C0463E480168C90703D1C8
:10192000016801220A4302607047C046012803D0C3
:10193000022809D1064800E00448364A13680340EB
:1019400013601068084310607047C046FFFFF1FF46
:10195000FF8FFFFFB0B5214B05280AD8052444436B
:101960000846A0401F25A5409C6AAC4304439C62E6
:101970001AE00B280BD8052444431E3C0846A0401F
:101980001F25A5405C6AAC4304435C620CE0102850
:101990000AD2052444433C3C0846A0401F25A540EC
:1019A0001C6AAC4304431C62092909D8032048433C
:1019B0008240072181405868884310435860B0BD79
:1019C000122909D8032048431E388240072181404C
:1019D0001868884310431860B0BDC0460C2401400D
:1019E00003210906234A13688B43136011680143DE
:1019F00011607047C107074904D0012292050B68A6
:101A000013430B60800704D5012040050A68024398
:101A10000A6070470824014040F200120346134058
:101A200091B1144913B10B6813430B60420504D5FF
:101A300040F200420B6813430B60800718D54868DA
:101A4000022202434A6070470A4923B10A6840F201
:101A500000139A430A60420504D50A6840F2004325
:101A60009A430A60800703D5486802229043486081
:101A70007047C04604240140142141433C480A58A1
:101A8000012313430B5070471421414338480A582F
:101A9000202313430B50704710B5142242430D49C5
:101AA000521853680124A34353600023536093608A
:101AB000D360136180000F228240086810430860E1
:101AC00010BDC04680008140024802680A4302609F
:101AD0007047C04604000240800081400248006810
:101AE0000840411E8841704700000240B0B51422F2
:101AF00042431F4813580124A343135013180C6882
:101B00009C608C68DC600C8A5C60135843F600743F
:101B1000A3434C681C43CB6823434C691C431450BB
:101B20000B7E5B1E5C425C41A30114584025AC4314
:101B3000E31813504B7E5B1E5C425C41E30114587A
:101B40008025AC43E3181350897E4B1E994109014F
:101B500013581024A34359181150B0BD1421414308
:101B600003480A5844F200039A430A507047C0469B
:101B70000800024010B5144608463F490A220A7080
:101B80000722214601F0D4FD012804D1044801F0C8
:101B900049FE012801D0032010BD002010BDC04621
:101BA000204E0000F8B506460F4CA088000A16D15A
:101BB000A0880527032810D30D460092A188264847
:101BC00001F030F948B9244908783070481C286081
:101BD000A088801E0099088000273846F8BD03A021
:101BE0000C499C22FFF746FEB40100207573526336
:101BF00076427566666572506F73203C204D425F79
:101C00005345525F5044555F53495A455F4D4158C3
:101C100000000000C03D0008B0B5174D6B780BB157
:101C2000052516E00124EC804B1EAB601870E88897
:101C30008018E880E988184601F0F4F8E9884A1C21
:101C4000EA80054A5054AC7000252846214601F030
:101C5000D1FB2846B0BDC046E80A002010B50120DF
:101C60000024214601F0C6FB03484470204610BC06
:101C700002BC8E4601F04ABDB401002080B50020B0
:101C8000014601F0B7FB80BC01BC864601F0E6BB13
:101C900010B5064C2078012805D10548806880479A
:101CA0000020207010BD062010BDC0460800002096
:101CB000F4010020F8B50C460988032505292FD129
:101CC0000279C17809028E18711E89B2314B99428E
:101CD00026D8811C00918778417800252580012332
:101CE000037023885B1C23805307B2B2D60803B16C
:101CF000761C009B46702088401C20800802C0197A
:101D0000401C81B218462B4600F0E8FA20B1F8BC1E
:101D100002BC8E4601F066B8F0B221880818208017
:101D20002846F8BDF8B50C460988032505292ED1AB
:101D30000279C17809028E18711E89B2154B994239
:101D400025D8811C009187784178002525800223C1
:101D5000037023885B1C23805307B2B2D60803B1FB
:101D6000761C009B46702088401C20800802C01909
:101D7000401C81B2184600F001FB20B1F8BC02BC47
:101D80008E4601F02FB8F0B221880818208028462E
:101D9000F8BDC046CE070000F8B50C4609880325FB
:101DA000052923D10279511E7C291FD8831C8178F3
:101DB000477800252580032606702688761C268015
:101DC000560046702088401C208038024018401C75
:101DD00081B218462B4600F0F7FA20B1F8BC02BCDD
:101DE0008E4600F0FFBF2088801920802846F8BD6D
:101DF000F8B50C4609880325052928D10179C27850
:101E0000120251184A1E92B27B2A20D8821C0092DC
:101E10008778437800252580042202702288521C8E
:101E200022808AB2560046702088401C208018020A
:101E3000C019401C81B2009800F0A2FB20B1F8BC90
:101E400002BC8E4600F0CEBF208880192080284634
:101E5000F8BDF8B5054608880A2841D30C4628790C
:101E6000E97809020F18781E80B203267C2838D83A
:101E7000287AE97909020818411E89B2782930D8F0
:101E8000697A82B2500081422BD1A879697909021E
:101E90000818411CA87800906E7828460A3089B24C
:101EA000012300F091FAB0B9BAB23002009940189B
:101EB000411CA81C0026268017232B7023885B1C3E
:101EC000238057006F7023885B1C238089B23346C0
:101ED00000F07AFA38B1F8BC02BC8E4600F082BF3E
:101EE00000263046F8BD2088C0192080F9E70000A0
:101EF000B0B50C4605490D88401C891C2A46FEF7E2
:101F00006FF9681C20800020B0BDC046C4010020CD
:101F10001CB50988032405291AD10179C1B9827831
:101F20004378C178FF2900D091B918028018421C6B
:101F300001A800244470FF394B424B41037091B219
:101F40000122134600F0CAF910B100F04BFF04461D
:101F500020461CBD80B50988052910D181784278BA
:101F600012025118491C89B2C01C0122134600F00C
:101F70002BFA30B180BC02BC8E4600F033BF032088
:101F800080BD002080BD70B50C460A880321062A5A
:101F900024D30679C27812029519AAB2D30876071B
:101FA00000D05B1C6D1EADB22D097A2D16D8457977
:101FB000DBB29D4212D1817843781B025918491C2B
:101FC00089B2801D012300F089F920B170BC02BCE8
:101FD0008E4600F007BF052020800021084670BD16
:101FE000B0B50C460A880321062A20D3027943792A
:101FF00055062D0EAB421AD1C3781B029A18531EF8
:102000009BB2772B13D8817843781B025918491C4F
:1020100089B2801D92B2012300F0D6F920B1B0BC84
:1020200002BC8E4600F0DEBE05202080002108465E
:10203000B0BD0000F8B50546022091B3CC081E2CB7
:102040002FD8069C524E3170012D15D04DBB254D19
:102050002548264FB760F0603561214870611F4800
:10206000B0611D48F0611B483062084611461A46AF
:10207000234600F091F813E0134D1448144FB76055
:10208000F06035610F4870610D48B0610B48F06138
:1020900009483062084611461A462346FFF76AFD92
:1020A00000B1F8BD01F02CFB20B1384801210170CE
:1020B0000020F8BD0320F8BDC9350008013600082E
:1020C000BD340008A51B0008191C00087D1C000871
:1020D0005D1C00080D390008593900087D380008DA
:1020E000D521000849220008C9220008AD220008B5
:1020F0007CB52648007808B1062445E001A801F027
:10210000F3FA002401283FD101A80078022812D058
:10211000012839D11E4D6B69681C294624312A1DBE
:10212000984788BB68782978884200D060BB022035
:1021300001F0ECFA28E0164D6A6A1178A9700023C4
:102140000120144C802B0AD0E65C46B18E4201D0AF
:102150000833F7E7E0184368291D10469847697867
:10216000002489B158B10121A980A97880220A43AD
:10217000696A0A70A9884A1CAA806A6A5054AA88A7
:10218000696A28782B69984720467CBD08000020A2
:10219000F40100200C00002010B514460846082267
:1021A000214601F0C5FA01280ED144F600308442E0
:1021B00001D9232003E060000549B1FBF0F080B2B3
:1021C00001F030FB012801D0032010BD002010BD1C
:1021D000A07F1700F8B506460F4C6088000A16D19C
:1021E00060880527042810D30D46009261882E4888
:1021F00001F018F848B92C4908783070481C28605C
:102200006088C01E0099088000273846F8BD03A0EA
:102210000C499C22FFF72EFBE801002075735263E6
:1022200076427566666572506F73203C204D425F42
:102230005345525F5044555F53495A455F4D41588D
:1022400000000000413E0008B0B51E4D2B78012B68
:1022500026D10124AC804B1EAB601870A888801872
:10226000A880A988184600F0DDFFA9884A1CAA802A
:102270000D4A5054A9884B1CAB80000A5054A868E2
:10228000007801F0C5FAA888401EA880A868401C04
:10229000A8606C7000252846214601F0ABF800E0EC
:1022A00005252846B0BDC046E80A002080B505488F
:1022B00000210170012001F09DF880BC01BC864620
:1022C00001F0E4B8E801002080B50020014601F0EB
:1022D00091F880BC01BC864601F0C0B8FEB514463A
:1022E0000246491E88B20019042824D8601E082519
:1022F000019590FBF5F0451C0020F3B1012B1BD19B
:1023000000901D4B280435D06D1E02921078224695
:10231000019F541E12040BD03A0609D0012202403C
:102320008EB29A55491C7F1EC0B240082246F0E783
:10233000029A521CE6E70120FEBD009008200190A1
:102340000D4F280416D002926D1E002622460198D9
:10235000541E12040AD0020608D08AB2BA5CB240F7
:102360001343761C491C401E2246F1E7029A137063
:10237000521CE6E70098FEBDE80B0020F0B5491EB0
:102380008BB2DC0801217D2C1BD39B1840F2EC346E
:10239000A34216D8511E082391FBF3F14C1C0021D7
:1023A00025040ED0641E16461D46721E360404D047
:1023B0006F1E2D0616463D46F7D100250570401CC0
:1023C000EEE70846F0BD0000FEB515460646481E7D
:1023D00087B20120604A974200D8A5E07A195F4C85
:1023E000A24200D9A0E041F27072BA1A5C4C62605D
:1023F000012B0CD023BB5848401C87425CD1022DD6
:102400005AD1500059490968564A115264E0019264
:10241000009065700522D24340F2D0735343514877
:10242000C3187C001B192C4622040BD032781202F0
:102430001A80707810181880B61C9B1C641EF3E775
:102440000020FEBD4448401C874247D1019840000F
:10245000444909182806C20D444C2046FDF7C0FE29
:10246000206808B1072801D30620206002AE307032
:1024700000240127204631463A46FEF79FF830787F
:102480003B4908700821081AFF21C140394D2970C5
:10249000384631463A46FEF765F8287802990140F9
:1024A00035484173314B186840F20072801818604B
:1024B000324801702046FEBD41F2A370081A303048
:1024C00080B2952831D85000264908189100274A33
:1024D00051186A00FDF784FE002227E041F2A37044
:1024E000081A80B2652800981ED8019840001D493E
:1024F00009181B48047866011B48871938460830BC
:102500002A06D20DFDF76CFE01201749885101986B
:102510007860601CC1B200221F291346114600D802
:1025200001460F4801701846FEBD01220520C04338
:1025300040F2D07141430B484018790040182904FB
:1025400007D04178317001787170B61C801C6D1E07
:10255000F5E71046FEBDC0466F170000581B00008F
:102560001C020020EC0B0020A006002080020020AE
:102570000100002000000020600200203002002046
:1025800010B50346481E81B20120084CA1420BD36E
:102590008918074CA14207D80020110404D05870B4
:1025A00018709B1C521EF8E710BDC046B80B000007
:1025B000BC0B0000FCB50191016A0090446A002543
:1025C0002E46202D0CD01746F740FF0705D0019F5F
:1025D000AF400F23AB40994339432D1D761CF0E7E4
:1025E00008250026202E0CD01346EB40DB0705D033
:1025F000019BB3400F27B740BC431C43361D6D1CE5
:10260000F0E7009801624462FCBD8162704781611D
:102610007047C162704700690840411E8841704799
:10262000FEB50293019202680090C5680026374605
:10263000202E10D0029BFB40DB0709D0019BB3404A
:102640000324B440A5431D430B46B340A2431A43A1
:10265000B61C7F1CECE700980260C560FEBDF8B5B3
:10266000012902D14168194301E041689943416061
:1026700000908168002403202646202C0CD01F46A1
:10268000F740FF0705D01746A7400546A540A943D8
:102690003943A41C761CF0E700988160F8BD000067
:1026A00096B00EA82021FDF7FAFDF24C00206082C2
:1026B000A0726072F049FF250D7007902070112004
:1026C000C0430B900C303C210A912A210991079AB2
:1026D00030B121180A9BCA54099BCA54401CF7E721
:1026E000FEF72CFFFFF79EF8FEF7EAF9FEF7A4FAD3
:1026F000FEF7C6F9FEF7A6F9FEF7E4F9FEF7AEFB22
:10270000FEF7EAFBFEF7BAFA41F2C020FEF744FBFF
:10271000FEF75CF9FEF7E6FCFEF738FC079EA661C3
:10272000FEF7A2FD01460096E12043023046324604
:10273000FFF780FCFFF7ACFADB4B58780A9960543E
:1027400040F2C811D94E715822463C32517340F2C2
:1027500000714118A18231600821081AC5401D701E
:1027600040F2D81030180B990C3151B1CD4A5218A3
:10277000036843241355036C49241355001D491C59
:10278000F3E7CB484021FFF740FFFEF707FC492362
:10279000C44AD05CC449097808400293D0541073ED
:1027A00001D0012090700798D072BF4CA0780840EB
:1027B000A070FDF7F8FFA078BA490874BB48343020
:1027C0006178079A19B102601030491EFAE70120BA
:1027D0000C9040F24810B54908180590B548C01C47
:1027E0000490B54844F20001FFF715FFAD4B0028F7
:1027F00000D1DDE0FFF77CFCAA49887940B1079859
:102800008871087A20B1012048210822FEF750FD86
:10281000AA48007800285BD00799A848017004985E
:10282000082914D08B000EAC0022E250E3181824C3
:102830001546042A07D0F8262640875CB7407D1944
:10284000F834521CF5E71D60001D491CE8E76421BF
:102850000E980D91B0FBF1F20A204243934CA26016
:102860002346C83328340025062D12D022600C9F41
:10287000AF408D498E7819688A4201D93E4302E003
:10288000374202D0BE4388498E7010341B1D6D1C28
:10289000EAE711990D9DB1FBF5F14143834A51617E
:1028A0000F99B1FBF5F141437E4AD4690B1B00221D
:1028B000A14200D213467D49CB601099B1FBF5F1DE
:1028C00048437849096A401A00D21046774908619E
:1028D000FDF7F0FF7A4F38B3FEF7FAFBFDF7BCFEC9
:1028E00000F0C2FB714C34346F484678E6B10B9867
:1028F00080000019406CFDF7CBFD7249FDF7D4FC58
:102900007149FDF7D1FC05462068FDF7C1FD014680
:10291000284601F061F8FDF777FD411C00D1002049
:1029200020601034761EE1E76849087800286CD0F2
:1029300000240C705D4D3035654F05980D90594B56
:102940005948407884422CD20B9880004619388828
:10295000FDF70CFF534B7064197881B10C99A140BD
:102960009A7B0D9B1B68984204D90A434D498A7390
:102970000B4604E01142F64B01D08A439A730A21B8
:10298000B0FBF1F0326CB2FBF1F24243B2FBF1F07A
:102990002860002001C710350D98001D0D90641CA3
:1029A000CEE7EC488078997B0143D973ED4F2EE058
:1029B000197BD87A08900D91884200D08AE0187867
:1029C000002800D1CDE0E6484178587B4840C0B2AD
:1029D000DA78002800D103E1002A00D116E10020B6
:1029E000D870DC4A12781A730A9A9A5C3633DB4C38
:1029F000002A00D126E10B9D585518705D192873E7
:102A0000A87101C4521E5B1CF2E7D14BD97B0806AA
:102A10000CD01A7CC8B290420FD01A7B8A431A732A
:102A2000FDF7C1FECA4BD87B187406E0187B1979F4
:102A3000014302D10298185C1873987A41017A58C0
:102A4000002A00D1C5E079184868412816D889685D
:102A50008000C14A11500A0EC14D43199F382A54B3
:102A60001A469C3A11701A469D3A0C0A14709E3B05
:102A7000A1E0C0462402002000000020512873D8A5
:102A800089688000B44A11500A0EB54D4319AF3819
:102A90002A541A46AC3A11701A46AD3A0C0A147010
:102AA000AE3B88E0240200200000002080020020CD
:102AB0000014004873010020000800487201002043
:102AC000A006002000007A44000061453C0100207F
:102AD000500100200A981C5C1879069098780390A1
:102AE00000259E4FAC4230D00D99E9400898E8404F
:102AF0005E192422B25C22BB0C9A1140104036228F
:102B0000B25CF2B93346243332463632884208D9B1
:102B100030200C9931540846069989B11870432029
:102B200008E00ED209980C9931540846039939B13E
:102B300018703D20305C40F2E8314843386000E0D6
:102B400010703F1D6D1C824BCCE7069808B1002029
:102B50001871039808B10020987002980D991954C3
:102B6000D9720C9818706FE0612811D889688000BC
:102B7000794A11500A0E7A4D4319BF382A541A4621
:102B8000BC3A11701A46BD3A0C0A1470BE3B12E0F2
:102B9000712829D8896880006F4A11500A0E704D3B
:102BA0004319CF382A541A46CC3A11701A46CD3AF6
:102BB0000C0A1470CE3B090C1970291880B204223B
:102BC000FDF7FCFC624B987A410100227A500C9987
:102BD000D971401CC1B21F2900D90020987200E6AB
:102BE00042B3002058802FE0972800D17AE0742863
:102BF00000D17CE0962800D180E0722800D084E0EB
:102C0000087A5449097801405973DCE75A79B2B11E
:102C10000020187358710A9A9A5C36334F4C8AB167
:102C20000B9D585518705D192873A87101C4521E68
:102C30005B1CF4E7587938B10020988004E0089ACA
:102C400050401873424B59730027444A0A98185C45
:102C5000874200D3CEE5DE193620305CD0B3304653
:102C60003630242100257554156005700C9CBC403D
:102C70000998305C0D9278B12A36F8B20121FEF73E
:102C800043FB334B344A40F2C8101158E0B20843BA
:102C900040F2C81150500EE03020305CE8B13036C0
:102CA000F8B22946FEF730FB294B2B4940F2C812F7
:102CB000885CA0438850357026490978014028482F
:102CC00041705973C9B20120FDF788FCFEF7BEFDC3
:102CD0001F4B0D9A121D7F1CB8E71F4840F2C81108
:102CE0004058E9E740F20110988000200BE0087A94
:102CF0001849097801401A48C17064E740F2011090
:102D000058801448007858735DE785280CD88A6885
:102D10000346713B1249CA54D1B284000E4D295169
:102D20000B4C001939380EE0952800D94BE78A681A
:102D30000346713B0A49CA54D1B28400064D295159
:102D4000034C00194338027098B2FDF747FC39E78D
:102D5000240200200000002080020020100100203A
:102D6000A0050020A006002070B540B2002817D4AE
:102D7000032302469A43144BD4588507ED0EFF26D1
:102D8000AE40B4438901C9B2A9402143D1501F21AB
:102D9000014001228A40400980000C49425070BD28
:102DA0008207D20EFF2494400F230340083B0320E8
:102DB000834304481D58A5438901C9B29140294362
:102DC000195070BD1CED00E000E400E000E100E0FF
:102DD000024A0A40024302480260704780FFFF1F18
:102DE00008ED00E040B1072803D0012803D10220FC
:102DF0007047062070470420704700000A2801D25F
:102E0000302102E0102803D237210818C0B27047E1
:102E100002A0034940F2D012FEF72CFD3000000062
:102E2000C03D000800220B0405D00378D218D2B2AE
:102E3000401C491EF7E75042C0B2704770490A680B
:102E40004CF200039A430A60CA6A2C4B1340CB62CF
:102E5000092851D8820001A39A18974600F012B8A9
:102E600000F015B800F01DB800F01EB800F01FB853
:102E700000F021B800F023B800F025B800F032B817
:102E800000F025B801200004CA6A824303E0012053
:102E90000004CA6A0243CA62C86A40F20012904340
:102EA00029E00868086022E00868086014E0086803
:102EB00044F2000219E0086844F200020AE00868DF
:102EC00048F2000211E0086848F2000202E00868D7
:102ED0004CF2000202430A600120C007CA6A0243A2
:102EE000CA6204E008684CF2000202430A60CA6A3F
:102EF00040F200101043C8627047C046FFFEFE7FDC
:102F0000F8B501463E4B18680C2202403D48082A9D
:102F1000044618D11A689202120F0F2A01D0941C8D
:102F200000E010241D682D0101D5113214461A68E5
:102F3000D20301D4344A05E09A6A0F2515406A1C71
:102F4000B0FBF2F254431D6818681A6805291FD8AF
:102F500000902D062D0F2DA77F5D2546FD40920484
:102F6000520F2E4FBE5C2A46F2408E0001A08019FF
:102F70008746C04600F00AB800F011B800F00AB861
:102F800000F00EB800F00EB800F014B8224607E0CA
:102F9000002205E000984005400F385CC5402A46F5
:102FA0001046F8BDD86AC0051AD4D86AC00320D527
:102FB0001C48F8BDD86A8007F2D0D86A03210840BF
:102FC00001282246ECD0D86A084048F200020228C4
:102FD000E6D0D86A084003280A4800D00020F8BD8F
:102FE00018680004800FD96A002904D4B2FBF0F2FB
:102FF000D6E70B48F8BD401CB5FBF0F2D0E7C04661
:103000000410024000127A0000093D000000000098
:10301000000000000102030406070809743D0008CF
:10302000809FD500003FAB011F21014001228A4053
:1030300080090C4943581343435070471F210140F6
:1030400001228A40800907494358934343507047FF
:103050001F21014001228A4080090249435813433D
:10306000435070470010024070B51348417803295F
:103070000BD8024614320023102B17D0C4186488D2
:1030800015682C1910C29B1CF6E7002141700246FE
:1030900014320A4B0C46102C0BD01D5B1668B60878
:1030A000751B00D20D4620C2A41CF4E7491C4170D8
:1030B00070BD0121017070BD3C0100206E02002036
:1030C0004162704710B5154C4449884213D01449E9
:1030D000884212D0EC49884211D03D49884213D031
:1030E0003D4988420DD03E4988420CD0394988423A
:1030F00013D1F63408E0E41D06E0F93404E0FD34B1
:1031000002E0641D00E0A41D2046FFF7A1FF204659
:1031100010BC02BC8E46FFF791BF10BD0B03000030
:10312000001000400168012291430160704701686E
:1031300001220A430260704710B50A888262244A5D
:10314000904202D0234B98420BD103687024A343D2
:1031500003604B8804681C4304608B8804681C432C
:1031600004608B68C36290420FD1136840F2003450
:10317000A3431360CB8814681C431460097B01636C
:10318000416901220A43426110BD124A90420BD0AC
:10319000C94A904208D0104A904205D00F4A904246
:1031A00002D00F4A9042EBD1026840F200339A43BA
:1031B0000260CA88036813430360074A9042DDD067
:1031C000074A9042DAD0054A9042D7D0D8E7C046A5
:1031D000002C014000040040004001400048014034
:1031E00000440140C2688A43C2607047C2680A4313
:1031F000C260704702698A4302617047C2680A4030
:10320000531E9A4100690840411E88411040704792
:103210000349002202730260426081607047C04629
:10322000FFFF0000F0B5FF24094A0A4B25460E04B3
:1032300009D006787540565D5F5D25467D40401C8F
:10324000491E3446F3E72002284380B2F0BDC04651
:10325000743C0008743B0008B0B50D4604467E4837
:10326000844204D02048844205D1022000E0052099
:10327000FFF746FE00E000202168090405D4690834
:103280004018B0FBF5F080B209E069084000401832
:10329000B0FBF5F0034901400007400F4018E06023
:1032A000B0BDC046F0FF0000416A034808407047C7
:1032B000014A0A4082627047FF01000010B566496A
:1032C000884204D0084988420BD1084C00E0054CE4
:1032D0002046FFF7BDFE204610BC02BC8E46FFF71D
:1032E000ADBE10BD0E0300000044004011040000FC
:1032F000016801220A43026070471F220A4001212F
:103300009140026A0A43026270471F220A408909FB
:103310000958D1400120084070471F220A4001236C
:10332000934089090A589A430A5070471F220A405D
:103330000123934089090A581A430A507047000034
:10334000084A914206D1D021425848F200039A43DC
:1033500042507047C902C90E01228A40016A1143D6
:103360000162704709340F341F220A400B049B0D81
:103370001B58D3408A0D1258C802C00EC2401A40D2
:10338000012010407047026801239A4302600268DE
:1033900040F200639A43026002680A430260704789
:1033A000026804239A43026002680A43026070477D
:1033B000026801239A430260426843F200039A4381
:1033C000426042680A4342607047026808239A4399
:1033D000026002680A4302607047026801239A4350
:1033E0000260026841F200039A43026002680A43E5
:1033F0000260704770B50E460921CC06CB4D052101
:10340000012808D12846FFF791FF204640F200111D
:10341000FFF7FBF807E02846FFF77FFF204640F262
:103420000011FFF7F4F806212846012E09D1FFF715
:103430007DFF204640F2001170BC04BC9646FFF7A9
:10344000E6B8FFF76AFF204640F2001170BC04BCEA
:103450009646FFF7DAB8C04600380140B0B5164CC2
:1034600000212046FFF72CFE012520462946FFF7C4
:10347000C1FE20462946FFF7B5FE2046B0BC02BC7F
:103480008E46FFF74FBEC04600200040B0B50A4C44
:1034900000212046FFF714FE012520462946FFF7AC
:1034A000A9FE20462946FFF7A1FE2046B0BC02BC7B
:1034B0008E46FFF73CBEC04600200040BCB53A4DEA
:1034C000A87800286AD101A800F028F968780024BB
:1034D00078B1022818D001285ED1FFF7D7FF01A8E4
:1034E00000780D2828D000243A2828D1EC70AC8030
:1034F00052E001A800783A284ED1FFF7C7FF002418
:10350000AC80EC70012018E001A80078297888428E
:1035100008D1FFF7A3FF00206870012000F0F6F843
:10352000044639E000243A2810D1EC70AC80012028
:103530006870FFF7ABFF2FE0022068702CE00146B7
:103540004139C9B2062903D3E14303E06C7023E09B
:10355000014637393038C2B20A2A00D30846E97822
:1035600001290AD0C1B9A988FF2911D8A988000169
:10357000E54A50540120E8700EE0A988E24A535C05
:1035800003435354A888401CA8800024EC7003E037
:1035900000246C70FFF762FF2046BCBD03A05149B8
:1035A000E322FEF767F9C046B401002065536E645C
:1035B0005374617465203D3D2053544154455F541C
:1035C000585F49444C45000080B53E484178491E4B
:1035D000012902D80021417005E04178012902D07B
:1035E0004078022803D1FFF739FF002080BD03484F
:1035F0003C4940F2A712FEF73DF9C0467C3D000869
:1036000070B5304E7078002856D1B078042840D874
:10361000810001A251188F4600F008B800F027B8C9
:1036200000F009B800F02BB800F014B80120002118
:10363000FFF7E0FE2DE0F08830B3F07801282AD0C3
:1036400038BBB06800780009FFF7D8FB00F0E0F85D
:10365000012012E00024B470032000F057F8054662
:1036600001202146FFF7C6FEB470284670BD3A20FF
:1036700000F0CEF80220B0700020F07009E0307841
:1036800000F0C6F8042003E00D2000F0C1F803208C
:10369000B070002070BDB06801780F200840FFF7BF
:1036A000ADFB00F0B5F80020F070B068401CB060D1
:1036B000F088401EF080ECE703A00A4940F24F1268
:1036C000FEF7D8F8B4010020655263765374617434
:1036D00065203D3D2053544154455F52585F494455
:1036E0004C450000C03D00080B490A78012A05D16D
:1036F0004A7802700020087001207047002070474F
:1037000005480021017001207047C04602494870F9
:10371000012008707047C046C001002010B5044663
:103720003F48FFF7C1FD2070012010BD0038014067
:10373000FEB502911B2000252946FFF715FB3148F5
:10374000FFF772FC0920C60601243046214640F2EC
:103750000022FEF72FFF022101913046224640F25F
:103760000023294FB847294F30462946224640F2C8
:103770000023B8473046214640F20042FEF71AFFC8
:1037800030460199224640F200431F4FB847304669
:103790002946224640F200431C4FB8473046214696
:1037A0002A4640F20013184FB847032230462946F4
:1037B00040F20013154EB0471248FD30FFF734FCBD
:1037C000174E3046FFF77AFD30460299FFF744FD69
:1037D00030462946FFF7ECFD30462946FFF7FDFD50
:1037E00030462946FFF7CFFD04213046FFF7D8FDCC
:1037F00008213046FFF7E9FD3046FFF779FD204606
:10380000FEBDC04611050000212600085F26000805
:1038100080B501460248FFF74BFD012080BDC04640
:10382000003801407FB5054640F20870FFF7FCFB09
:10383000104C2046FFF746FC6E463046FFF7E8FC8A
:103840000D483080681E02900020019020463146CD
:10385000FFF772FC012520462946FFF7C7FC13201D
:103860002946FFF781FA2046FFF761FC284604B09D
:1038700070BDC046002000400F0E00001CB51A4C61
:10388000607858BB01A8FFF749FF2078032823D8A8
:10389000810001A251188F4600F01CB800F004B856
:1038A00000F00CB800F016B8002060806088411C61
:1038B00061801549019A0A5402200AE06088FF28B5
:1038C00006D86088411C61800F49019A0A5401E0C2
:1038D00003202070FFF7DAFD00201CBD03A03D4946
:1038E000F022FDF7C7FFC046E801002065536E6473
:1038F0005374617465203D3D2053544154455F54D9
:10390000585F49444C450000E80A0020B0B5294DF5
:1039100028780024032808D0022802D058B90020B3
:1039200000E00120FFF7F2FE0446FFF797FD0120BB
:1039300028702046B0BD28780028F6D028780228C4
:10394000F3D028780328F0D00248224940F26512CB
:10395000FDF790FFDE3D000870B5164E3078012867
:1039600022D17078012805D080B901200021FFF70D
:1039700041FD0BE0B08858B1B0680078FFF748FF10
:10398000B068401CB060B088401EB080002070BDA0
:103990000320FFF7BBFE0446012000252946FFF760
:1039A00029FD7570204670BD03A00A4940F22B1214
:1039B000FDF760FFE801002065526376537461747F
:1039C00065203D3D2053544154455F52585F494462
:1039D0004C450000413E000870B50125ED0704008C
:1039E0004C4020D4441A01D2001B0919C60D4B00CB
:1039F000F2B2FF2A29D01B0E2CD000020C02284361
:103A00002C43D31ADC40051910D2280A02D3401CDB
:103A10006D0611D0761EF6058019FF2A00DA70BDFA
:103A2000C00DC00570BD694000F022F801200543BB
:103A3000C541521C761CE8E764089C40C9016140FE
:103A40008900E7D10124A043E4E71B0E440200D023
:103A5000034870BD002AFCD1C00FC00770BD00BF75
:103A60000000C07F70B50125ED0704004C4022D452
:103A7000441A02D26C40001B0919C60D4B00F2B269
:103A8000FF2A4BD01B0E50D000020C02A8432C433F
:103A9000D31ADC40051B05D5AD0019D36D08761E81
:103AA000521E37D0F605280A01D2801970BD704128
:103AB0006D0603D070BD6940FFF794FF9C4009027A
:103AC0006140490001D0401E70BD0124A04370BD7B
:103AD0006D081DD001202B0C01D12D0410302B0EB0
:103AE00001D12D0208302B0F01D12D01001DAB0F8C
:103AF00001D1AD00801CEB0F01D16D00401C361AC6
:103B0000121A6D00680AF5054019012A02DB70BD22
:103B1000002070BDC036300AC00770BD1B0E4402C5
:103B200001D1FF2B00D1024870BD002AF0D070BD3A
:103B30000000C07F8182838485868788898B8C8DF5
:103B40008E8F919293959697999A9C9D9FA0A2A3F0
:103B5000A5A7A8AAACAEB0B2B3B5B7B9BCBEC0C237
:103B6000C5C7C9CCCED1D4D7D9DCDFE2E6E9ECF0C9
:103B7000F3F7FAFE00C1814001C0804101C08041DD
:103B800000C1814001C0804100C1814000C181402D
:103B900001C0804101C0804100C1814000C181401D
:103BA00001C0804100C1814001C0804101C080410D
:103BB00000C1814001C0804100C1814000C18140FD
:103BC00001C0804100C1814001C0804101C08041ED
:103BD00000C1814000C1814001C0804101C08041DD
:103BE00000C1814001C0804100C1814000C18140CD
:103BF00001C0804101C0804100C1814000C18140BD
:103C000001C0804100C1814001C0804101C08041AC
:103C100000C1814000C1814001C0804101C080419C
:103C200000C1814001C0804100C1814000C181408C
:103C300001C0804100C1814001C0804101C080417C
:103C400000C1814001C0804100C1814000C181406C
:103C500001C0804101C0804100C1814000C181405C
:103C600001C0804100C1814001C0804101C080414C
:103C700000C1814000C0C101C30302C2C60607C71C
:103C800005C5C404CC0C0DCD0FCFCE0E0ACACB0B8C
:103C9000C90908C8D81819D91BDBDA1A1EDEDF1FBC
:103CA000DD1D1CDC14D4D515D71716D6D21213D3AC
:103CB00011D1D010F03031F133F3F23236F6F7375C
:103CC000F53534F43CFCFD3DFF3F3EFEFA3A3BFB4C
:103CD00039F9F83828E8E929EB2B2AEAEE2E2FEFFC
:103CE0002DEDEC2CE42425E527E7E62622E2E3236C
:103CF000E12120E0A06061A163A3A26266A6A7679C
:103D0000A56564A46CACAD6DAF6F6EAEAA6A6BAB0B
:103D100069A9A86878B8B979BB7B7ABABE7E7FBF3B
:103D20007DBDBC7CB47475B577B7B67672B2B3732B
:103D3000B17170B0509091519353529296565797DB
:103D4000559594549C5C5D9D5F9F9E5E5A9A9B5BCB
:103D500099595898884849894B8B8A4A4E8E8F4F7B
:103D60008D4D4C8C448485458747468682424383EB
:103D700041818040000000000102030428206552B8
:103D800063765374617465203D3D2053544154451E
:103D90005F52585F5243562029207C7C20282065A2
:103DA0005263765374617465203D3D2053544154F1
:103DB000455F52585F574149545F454F462029009F
:103DC0002E2E2F4170702F4D6F646275732F6173AB
:103DD0006369692F6D6261736369692E63002820CE
:103DE000655263765374617465203D3D20535441A0
:103DF00054455F52585F494E49542029207C7C200D
:103E00002820655263765374617465203D3D2053CC
:103E1000544154455F52585F5243562029207C7CC0
:103E2000202820655263765374617465203D3D20DF
:103E300053544154455F52585F4552524F522029C6
:103E4000002E2E2F4170702F4D6F646275732F728C
:103E500074752F6D627274752E630000803E0008C9
:103E6000000000209000000010010008103F000832
:103E700090000020301B00002C0100080000000012
:103E8000FF06FF0000A24A0402000000110000002B
:103E9000F11E000804000000F11D000803000000EE
:103EA000991D000810000000E11F00080600000036
:103EB000551F000817000000531E000801000000F5
:103EC000B51C000805000000111F00080F000000CD
:103ED000871F000802000000251D000800000000E8
:103EE00000000000000000000000000000000000D2
:103EF00000000000000000000000000000000000C2
:103F000000000000000000000000000000000000B1
:04000005080000CD22
:00000001FF
